:1000000012C02CC02BC02AC029C028C027C026C0BF
:1000100025C024C023C022C021C020C01FC01EC0D4
:100020001DC01CC01BC011241FBECFE5D4E0DEBF25
:10003000CDBF10E0A0E6B0E0E2EAF8E102C0059032
:100040000D92AE3EB107D9F710E0AEEEB0E001C0C0
:100050001D92AF3FB107E1F799D421CCD1CF0895DC
:10006000AD988FEF82BBAD9A08951F93CF93DF9326
:10007000EC011FEF25C08091FD0082BBAD98AC98CC
:1000800012BBAD9A8091F00082BBEADF8091F9004B
:1000900082BBE6DF8091FC0082BBE2DF8091FE0044
:1000A00082BBDEDF8091F20082BBDADF8091F40058
:1000B00082BBD6DF8091F60082BBD2DFAC9A21975B
:1000C0002097C9F6DF91CF911F91089581E090E0CC
:1000D00008C081E090E0C9DF8091F7009091F800BE
:1000E00001969093F8008093F7002091F7003091EB
:1000F000F8008091EC009091ED00281739074CF33F
:100100008091F4008093F6008091F2008093F400D7
:100110008091FE008093F2008091FC008093FE00AD
:100120008091F9008093FC008091F0008093F900A9
:100130008091FD008093F0000895AF92BF92CF921E
:10014000DF92EF92FF920F931F93A090FD00B0906B
:10015000F000C090F900D090FC00E090FE00F0901C
:10016000F2000091F4001091F600F0916900A09166
:10017000680070916700B0916600509165006091D1
:100180006400E091630040916200909161002091D1
:10019000600031E04FC0213011F4492F1BC02230E4
:1001A00011F4E92F17C0233011F4692F13C0243044
:1001B00011F4592F0FC0253011F4B92F0BC0263080
:1001C00011F4792F07C0273011F4A92F03C028306C
:1001D00009F4F92F842F8A298F3FE1F48E2F8B2980
:1001E0008F3FC1F4862F8C298F3FA1F4852F8D2955
:1001F0008F3F81F48B2F8E298F3F61F4872F8F29BA
:100200008F3F41F48A2F802B8F3F21F48F2F812B3A
:100210008F3F99F03F5F990F91609F3F09F49EEFE8
:100220003A3040F02F5F293010F431E0B4CF21E0B4
:1002300031E0B3CF332309F0AECFF0936900A09340
:10024000680070936700B0936600509365006093F8
:100250006400E093630040936200909361002093F8
:1002600060001092F1001F910F91FF90EF90DF90CE
:10027000CF90BF90AF900895EF92FF920F931F938E
:10028000EE24EA94E092FD0021DF8FE1F82EF09257
:10029000FD001CDF03E00093FD0018DF1CEC109351
:1002A000FD0014DF1093FD0011DF0093FD000EDF51
:1002B000F092FD000BDFE092FD0008DF1F910F912F
:1002C000FF90EF9008951F931FEF1093FD00FEDE47
:1002D0001092FD00FBDE1092FD00F8DE8CE38093AF
:1002E000FD00F4DE84E28093FD00F0DE1092FD005C
:1002F000EDDE89E98093FD00E9DE1093FD00E6DE86
:100300001F9108950F931F930FEF0093FD00DEDE02
:1003100081E88093FD00DADE1092FD00D7DE1CE359
:100320001093FD00D3DE1093FD00D0DE88E18093B2
:10033000FD00CCDE89E98093FD00C8DE0093FD005E
:10034000C5DE1F910F9108950F931F930FEF009338
:10035000FD00BCDE1092FD00B9DE1092FD00B6DE9D
:100360001CE31093FD00B2DE1093FD00AFDE10928F
:10037000FD00ACDE81E88093FD00A8DE0093FD0067
:10038000A5DE1F910F9108950F931F930FEF009318
:10039000FD009CDE1092FD0099DE1092FD0096DEBD
:1003A00014E21093FD0092DE1093FD008FDE109397
:1003B000FD008CDE8CE38093FD0088DE0093FD0061
:1003C00085DE1F910F9108950F931F930FEF0093F8
:1003D000FD007CDE1092FD0079DE1092FD0076DEDD
:1003E00014EE1093FD0072DE1093FD006FDE10938B
:1003F000FD006CDE8CEF8093FD0068DE0093FD0055
:1004000065DE1F910F9108951F931FEF1093FD005C
:100410005DDE81E88093FD0059DE1092FD0056DE1E
:100420008CE38093FD0052DE8CE28093FD004EDE73
:1004300088E08093FD004ADE89E88093FD0046DE77
:100440001093FD0043DE1F9108950F931F930FEF4C
:100450000093FD003BDE1092FD0038DE1092FD009F
:1004600035DE17EE1093FD0031DE1093FD002EDE19
:100470001092FD002BDE1092FD0028DE0093FD009F
:1004800025DE1F910F9108950F931F930FEF009397
:10049000FD001CDE1CE31093FD0018DE1092FD0031
:1004A00015DE1092FD0012DE1093FD000FDE0093AA
:1004B000FD000CDE1F910F9108950F931F930FEF16
:1004C0000093FD0003DE8CE98093FD00FFDD8CE1ED
:1004D0008093FD00FBDD1CE31093FD00F7DD10931E
:1004E000FD00F4DD1092FD00F1DD80E88093FD0059
:1004F000EDDD0093FD00EADD1F910F9108951F933C
:100500001FEF1093FD00E2DD1092FD00DFDD109281
:10051000FD00DCDD83EC8093FD00D8DD81E8809375
:10052000FD00D4DD88E18093FD00D0DD8CE3809375
:10053000FD00CCDD1093FD00C9DD1F9108950F93E0
:100540001F930FEF0093FD00C1DD1092FD00BEDD93
:100550001092FD00BBDD1FE31093FD00B7DD10938B
:10056000FD00B4DD1093FD00B1DD1093FD00AEDDA4
:100570000093FD00ABDD1F910F910895FF920F9343
:100580001F93FF24FA94F092FD00A0DD1092FD006D
:100590009DDD1092FD009ADD09EF0093FD0096DDD0
:1005A00013EF1093FD0092DD1093FD008FDD00939B
:1005B000FD008CDD1092FD0089DD1092FD0086DDCE
:1005C000F092FD0083DD1F910F91FF9008951F931E
:1005D0001FEF1093FD007ADD1092FD0077DD109281
:1005E000FD0074DD81EF8093FD0070DD83EE80936C
:1005F000FD006CDD87EC8093FD0068DD8FE8809363
:10060000FD0064DD1092FD0061DD1092FD005EDDF5
:100610001093FD005BDD1F910895FF920F931F93D0
:10062000FF24FA94F092FD0051DD01E80093FD00F3
:100630004DDD1092FD004ADD1CE31093FD0046DD08
:100640001093FD0043DD1092FD0040DD0093FD009E
:100650003DDDF092FD003ADD1F910F91FF9008956E
:100660000F931F930FEF0093FD0030DD1092FD00FC
:100670002DDD1092FD002ADD14EE1093FD0026DD25
:100680001093FD0023DD80EE8093FD001FDD81EFE0
:100690008093FD001BDD0093FD0018DD1F910F917D
:1006A00008951F931FEF1093FD0010DD81E88093E4
:1006B000FD000CDD1092FD0009DD8CE28093FD0051
:1006C00005DD8CE18093FD0001DD1092FD00FEDC74
:1006D00081E08093FD00FADC1093FD00F7DC1F91B0
:1006E00008951F931FEF1093FD00F0DC1092FD00A2
:1006F000EDDC1092FD00EADC84EC8093FD00E6DC8A
:1007000084E88093FD00E2DC80E28093FD00DEDC83
:1007100081E78093FD00DADC1093FD00D7DC1F91A8
:1007200008950F931F930FEF0093FD00CFDC81E935
:100730008093FD00CBDC80E38093FD00C7DC14E2F6
:100740001093FD00C3DC1093FD00C0DC8CE08093AF
:10075000FD00BCDC89E88093FD00B8DC0093FD005F
:10076000B5DC1F910F9108950F931F930FEF009326
:10077000FD00ACDC1CEF1093FD00A8DC1093FD0025
:10078000A5DC1092FD00A2DC1092FD009FDC10930E
:10079000FD009CDC1093FD0099DC0093FD0096DCCD
:1007A0001F910F910895FF920F931F93FF24FA94C6
:1007B000F092FD008BDC00E80093FD0087DC1092D6
:1007C000FD0084DC1FE31093FD0080DC1093FD002E
:1007D0007DDC1092FD007ADC0093FD0077DCF09266
:1007E000FD0074DC1F910F91FF900895EF92FF922E
:1007F0000F931F93EE24EA94E092FD0067DC90EFE4
:10080000F92EF092FD0062DC00EC0093FD005EDC4E
:100810001FE01093FD005ADC1093FD0057DC00939D
:10082000FD0054DCF092FD0051DCE092FD004EDC56
:100830001F910F91FF90EF900895FF920F931F93D8
:10084000FF24FA94F092FD0041DC1092FD003EDCA2
:100850001092FD003BDC0FE90093FD0037DC1FEC3C
:100860001093FD0033DC1093FD0030DC0093FD009D
:100870002DDC1092FD002ADC1092FD0027DCF092A6
:10088000FD0024DC1F910F91FF900895EF92FF92DD
:100890000F931F93EE24EA94E092FD0017DC2CE303
:1008A000F22EF092FD0012DC08E10093FD000EDC58
:1008B00013EC1093FD000ADC1093FD0007DC00939D
:1008C000FD0004DCF092FD0001DCE092FD00FEDBA7
:1008D0001F910F91FF90EF900895EF92FF920F9369
:1008E0001F93EE24EA94E092FD00F0DB3CEFF32E40
:1008F000F092FD00EBDB00EF0093FD00E7DB13E07F
:100900001093FD00E3DB1093FD00E0DB0093FD009E
:10091000DDDBF092FD00DADBE092FD00D7DB1F911A
:100920000F91FF90EF9008951F931FEF1093FD001C
:10093000CDDB8CE18093FD00C9DB8CE08093FD0072
:10094000C5DB84E08093FD00C1DB80E28093FD0085
:10095000BDDB80E38093FD00B9DB88E38093FD007D
:10096000B5DB1093FD00B2DB1F9108951F931FEFBD
:100970001093FD00ABDB1093FD00A8DB1093FD008E
:10098000A5DB1093FD00A2DB1F910895BF92CF92CB
:10099000DF92EF92FF920F931F931FEF11BB80E343
:1009A00084BB8FEC85BB1093F6001093F40010937A
:1009B000F2001093FE001093FC001093F9001093C6
:1009C000F0001093FD00ADDE02DE56DC98DDDCDCCD
:1009D000CDDFCCDF1093F6001093F4001093F200FB
:1009E0001093FE001093FC001093F9001093F00098
:1009F0001093FD00A2DBEE24E39474E0C72E63E0C5
:100A0000B62E52E0D52E1EEF0FEF4FE7F42E809159
:100A1000EF00823051F4989B08C0999B06C09A9BC6
:100A200004C09B9B02C01092EF008091EF008823CE
:100A300009F046C080916100880F81608093610059
:100A40008F3F11F41093610098990DC08091EB00D5
:100A5000813011F0833019F4D092EB0002C0B092D3
:100A6000EB00E092EF0099990DC08091EB0081308E
:100A700011F0833019F4D092EB0002C0E092EB0049
:100A8000E092EF009A990DC08091EB00813011F057
:100A9000833019F4C092EB0002C0B092EB00E092F8
:100AA000EF009B990DC08091EB00813011F08330F5
:100AB00019F4C092EB0002C0E092EB00E092EF006C
:100AC0008091EE00843608F4E1C6809160008F5F6B
:100AD00080936000893010F0E09260008091EB001C
:100AE000813009F058C080916A008E3F19F4F0926D
:100AF0006A0004C08695806880936A0080916B00CC
:100B00008E3F19F4F0926B0004C086958068809344
:100B10006B0080916C008E3F19F4F0926C0004C061
:100B20008695806880936C0080916D008E3F19F4EB
:100B3000F0926D0004C08695806880936D0080916E
:100B40006E008E3F19F4F0926E0004C086958068A6
:100B500080936E0080916F008E3F19F4F0926F00C9
:100B600004C08695806880936F00809170008E3FEE
:100B700019F4F092700004C086958068809370002C
:100B8000809171008E3F19F4F092710004C0869537
:100B90008068809371008091EB00823011F5909114
:100BA0006A009093F30080916B0080936A008091BB
:100BB0006C0080936B0080916D0080936C0080913D
:100BC0006E0080936D0080916F0080936E00809125
:100BD000700080936F0080917100809370009093FB
:100BE00071008091EB00833009F058C080916A0059
:100BF0008F3719F410936A0004C0880F81608093C6
:100C00006A0080916B008F3719F410936B0004C059
:100C1000880F816080936B0080916C008F3719F48E
:100C200010936C0004C0880F816080936C008091E9
:100C30006D008F3719F410936D0004C0880F816028
:100C400080936D0080916E008F3719F410936E00C1
:100C500004C0880F816080936E0080916F008F3791
:100C600019F410936F0004C0880F816080936F00A7
:100C7000809170008F3719F41093700004C0880FB2
:100C8000816080937000809171008F3719F4109308
:100C9000710004C0880F8160809371008091EB0027
:100CA000843011F5909171009093F3008091700061
:100CB0008093710080916F008093700080916E002E
:100CC00080936F0080916D0080936E0080916C0026
:100CD00080936D0080916B0080936C0080916A001E
:100CE00080936B0090936A001092EE00D092EF0018
:100CF00020916A0080916200281709F041C090910C
:100D00006B00809163009817D9F590916C008091E9
:100D100064009817A9F590916D008091650098176F
:100D200079F590916E0080916600981749F5909141
:100D30006F0080916700981719F59091700080916D
:100D400068009817E9F490917100809169009817F4
:100D5000B9F4009369000093680000936700009362
:100D600066000093650000936400009363000093A5
:100D700062008091EA008F5F8093EA00DED942C072
:100D80008091FD00282B2F3F89F580916B00909179
:100D9000F000892B8F3F51F580916C009091F90004
:100DA000892B8F3F19F580916D009091FC00892B64
:100DB0008F3FE1F480916E009091FE00892B8F3F70
:100DC000A9F480916F009091F200892B8F3F71F40C
:100DD000809170009091F400892B8F3F39F48091BD
:100DE00071009091F600892B8F3F61F00DDB44DAA2
:100DF000C5DBCADABBDD11DCF9DCC6DA72DCB6DDD4
:100E0000B5DDF4CFE091720080916A00E823809113
:100E10007A00E82380916200E823E093FD0070915E
:100E2000730080916B00782380917B007823809100
:100E3000630078237093F0006091740080916C00DF
:100E4000682380917C00682380916400682360930C
:100E5000F9005091750080916D00582380917D00BC
:100E600058238091650058235093FC0040917600F0
:100E700080916E00482380917E0048238091660017
:100E800048234093FE003091770080916F00382313
:100E900080917F0038238091670038233093F200DF
:100EA0002091780080917000282380918000282371
:100EB0008091680028232093F4009091790080911C
:100EC0007100982380918100982380916900982374
:100ED0009093F6008091EA00843040F18091820086
:100EE000E823E093FD008091830078237093F00065
:100EF0008091840068236093F900809185005823D5
:100F00005093FC008091860048234093FE0080911E
:100F1000870038233093F2008091880028232093A3
:100F2000F4008091890098239093F6008091EA0064
:100F30008530C0F18091FD0090918A0089238093D3
:100F4000FD008091F00090918B0089238093F00048
:100F50008091F90090918C0089238093F900809111
:100F6000FC0090918D0089238093FC008091FE000D
:100F700090918E0089238093FE008091F2009091E1
:100F80008F0089238093F2008091F400909190006B
:100F900089238093F4008091F60090919100892339
:100FA0008093F6008091EA008630C0F18091FD00C8
:100FB0009091920089238093FD008091F0009091A0
:100FC000930089238093F0008091F9009091940020
:100FD00089238093F9008091FC00909195008923EA
:100FE0008093FC008091FE0090919600892380936D
:100FF000FE008091F2009091970089238093F20087
:101000008091F4009091980089238093F40080915E
:10101000F6009091990089238093F6008091EA0070
:101020008730C0F18091FD0090919A0089238093D0
:10103000FD008091F00090919B0089238093F00047
:101040008091F90090919C0089238093F900809110
:10105000FC0090919D0089238093FC008091FE000C
:1010600090919E0089238093FE008091F2009091E0
:101070009F0089238093F2008091F4009091A0005A
:1010800089238093F4008091F6009091A100892338
:101090008093F6008091EA008830C0F18091FD00D5
:1010A0009091A20089238093FD008091F00090919F
:1010B000A30089238093F0008091F9009091A4000F
:1010C00089238093F9008091FC009091A5008923E9
:1010D0008093FC008091FE009091A600892380936C
:1010E000FE008091F2009091A70089238093F20086
:1010F0008091F4009091A80089238093F40080915E
:10110000F6009091A90089238093F6008091EA006F
:101110008930C0F18091FD009091AA0089238093CD
:10112000FD008091F0009091AB0089238093F00046
:101130008091F9009091AC0089238093F90080910F
:10114000FC009091AD0089238093FC008091FE000B
:101150009091AE0089238093FE008091F2009091DF
:10116000AF0089238093F2008091F4009091B00049
:1011700089238093F4008091F6009091B100892337
:101180008093F6008091EA008A30C0F18091FD00E2
:101190009091B20089238093FD008091F00090919E
:1011A000B30089238093F0008091F9009091B400FE
:1011B00089238093F9008091FC009091B5008923E8
:1011C0008093FC008091FE009091B600892380936B
:1011D000FE008091F2009091B70089238093F20085
:1011E0008091F4009091B80089238093F40080915D
:1011F000F6009091B90089238093F6008091EA006F
:101200008B30C0F18091FD009091BA0089238093CA
:10121000FD008091F0009091BB0089238093F00045
:101220008091F9009091BC0089238093F90080910E
:10123000FC009091BD0089238093FC008091FE000A
:101240009091BE0089238093FE008091F2009091DE
:10125000BF0089238093F2008091F4009091C00038
:1012600089238093F4008091F6009091C100892336
:101270008093F6008091EA008C30C0F18091FD00EF
:101280009091C20089238093FD008091F00090919D
:10129000C30089238093F0008091F9009091C400ED
:1012A00089238093F9008091FC009091C5008923E7
:1012B0008093FC008091FE009091C600892380936A
:1012C000FE008091F2009091C70089238093F20084
:1012D0008091F4009091C80089238093F40080915C
:1012E000F6009091C90089238093F6008091EA006E
:1012F0008D30C0F18091FD009091CA0089238093C8
:10130000FD008091F0009091CB0089238093F00044
:101310008091F9009091CC0089238093F90080910D
:10132000FC009091CD0089238093FC008091FE0009
:101330009091CE0089238093FE008091F2009091DD
:10134000CF0089238093F2008091F4009091D00027
:1013500089238093F4008091F6009091D100892335
:101360008093F6008091EA008E30C0F18091FD00FC
:101370009091D20089238093FD008091F00090919C
:10138000D30089238093F0008091F9009091D400DC
:1013900089238093F9008091FC009091D5008923E6
:1013A0008093FC008091FE009091D6008923809369
:1013B000FE008091F2009091D70089238093F20083
:1013C0008091F4009091D80089238093F40080915B
:1013D000F6009091D90089238093F6008091EA006D
:1013E0008F30C0F18091FD009091DA0089238093C5
:1013F000FD008091F0009091DB0089238093F00044
:101400008091F9009091DC0089238093F90080910C
:10141000FC009091DD0089238093FC008091FE0008
:101420009091DE0089238093FE008091F2009091DC
:10143000DF0089238093F2008091F4009091E00016
:1014400089238093F4008091F6009091E100892334
:101450008093F6008091EA008031C0F18091FD0018
:101460009091E20089238093FD008091F00090919B
:10147000E30089238093F0008091F9009091E400CB
:1014800089238093F9008091FC009091E5008923E5
:101490008093FC008091FE009091E6008923809368
:1014A000FE008091F2009091E70089238093F20082
:1014B0008091F4009091E80089238093F40080915A
:1014C000F6009091E90089238093F6008091DA007C
:1014D0008093E2008091DB008093E3008091DC0048
:1014E0008093E4008091DD008093E5008091DE0030
:1014F0008093E6008091DF008093E7008091E00018
:101500008093E8008091E1008093E9008091D2000F
:101510008093DA008091D3008093DB008091D40027
:101520008093DC008091D5008093DD008091D6000F
:101530008093DE008091D7008093DF008091D800F7
:101540008093E0008091D9008093E1008091CA00EF
:101550008093D2008091CB008093D3008091CC0007
:101560008093D4008091CD008093D5008091CE00EF
:101570008093D6008091CF008093D7008091D000D7
:101580008093D8008091D1008093D9008091C200CF
:101590008093CA008091C3008093CB008091C400E7
:1015A0008093CC008091C5008093CD008091C600CF
:1015B0008093CE008091C7008093CF008091C800B7
:1015C0008093D0008091C9008093D1008091BA00AF
:1015D0008093C2008091BB008093C3008091BC00C7
:1015E0008093C4008091BD008093C5008091BE00AF
:1015F0008093C6008091BF008093C7008091C00097
:101600008093C8008091C1008093C9008091B2008E
:101610008093BA008091B3008093BB008091B400A6
:101620008093BC008091B5008093BD008091B6008E
:101630008093BE008091B7008093BF008091B80076
:101640008093C0008091B9008093C1008091AA006E
:101650008093B2008091AB008093B3008091AC0086
:101660008093B4008091AD008093B5008091AE006E
:101670008093B6008091AF008093B7008091B00056
:101680008093B8008091B1008093B9008091A2004E
:101690008093AA008091A3008093AB008091A40066
:1016A0008093AC008091A5008093AD008091A6004E
:1016B0008093AE008091A7008093AF008091A80036
:1016C0008093B0008091A9008093B10080919A002E
:1016D0008093A20080919B008093A30080919C0046
:1016E0008093A40080919D008093A50080919E002E
:1016F0008093A60080919F008093A7008091A00016
:101700008093A8008091A1008093A900809192000D
:1017100080939A008091930080939B008091940025
:1017200080939C008091950080939D00809196000D
:1017300080939E008091970080939F0080919800F5
:101740008093A000809199008093A10080918A00ED
:101750008093920080918B008093930080918C0005
:101760008093940080918D008093950080918E00ED
:101770008093960080918F008093970080919000D5
:1017800080939800809191008093990080918200CD
:1017900080938A008091830080938B0080918400E5
:1017A00080938C008091850080938D0080918600CD
:1017B00080938E008091870080938F0080918800B5
:1017C00080939000809189008093910080917A00AD
:1017D0008093820080917B008093830080917C00C5
:1017E0008093840080917D008093850080917E00AD
:1017F0008093860080917F00809387008091800095
:10180000809388008091810080938900809172008C
:1018100080937A008091730080937B0080917400A4
:1018200080937C008091750080937D00809176008C
:1018300080937E008091770080937F008091780074
:1018400080938000809179008093810080916A006C
:101850008093720080916B008093730080916C0084
:101860008093740080916D008093750080916E006C
:101870008093760080916F00809377008091700054
:101880008093780080917100809379008EE190E0E0
:10189000ECD38091EE008F5F8093EE00B8C8F8948F
:0218A000FFCF78
:1018A20002FBFFFFFFFFFFFFFFFFEFFFFFFFFFFF57
:1018B200FFFFFFFFFFFFFFFFFFFFFFFFFFFFFFFF36
:1018C200FFFFFFFFFFFFFFFFFFFFFFFFFFFFFFFF26
:1018D200FFFFFFFFFFFFFFFFFFFFFFFFFFFFFFFF16
:1018E200FFFFFFFFFFFFFFFFFFFFFFFFFFFFFFFF06
:1018F200FFFFFFFFFFFFFFFFFFFFFFFFFFFFFFFFF6
:10190200FFFFFFFFFFFFFFFFFFFFFFFFFFFFFFFFE5
:10191200FFFFFFFFFFFFFFFFFFFFFFFFFFFFFFFFD5
:0E192200FFFFFFFFFFFFFFFFFFFF0302580262
:00000001FF
